:100000000C9496000C94B5000C94B5000C94B500BB
:100010000C94B5000C94B5000C94B5000C94B5008C
:100020000C94B5000C94B5000C94D9020C94B50056
:100030000C94B5000C94B5000C94B5000C94B5006C
:100040000C94B5000C94B5000C94B5000C94B5005C
:100050000C94B5000C94B5000C94B5000C94B5004C
:100060000C94B5000C94B5000C94B5000C94B5003C
:100070000C94B5000C94B5000C94B5000C94B5002C
:100080000C94B5000C94B5000C94B5000C94B5001C
:100090000C94B5000C94B50012010002020000405F
:1000A000EB031820001000000001090243000201C8
:1000B0000080320904000001020201000524001042
:1000C000010524010301042402060524060001079A
:1000D0000583032000FF09040100020A0000000755
:1000E000058102200000070502022000000C0341E8
:1000F0000054004D0045004C0022034100560052C0
:1001000000200055005300420020004300440043FB
:10011000002000440045004D004F000C0331002E2C
:100120000030002E003000040309040011241FBE1B
:10013000CFEFD0E2DEBFCDBF11E0A0E0B1E0E0E163
:10014000F1E100E00BBF02C007900D92A037B107AC
:10015000D9F711E0A0E7B1E001C01D92A339B107C2
:10016000E1F70E9425020C9486080C94000080E0C0
:1001700008958091E800877F8093E800809178015E
:100180008093F100809179018093F10080917A0150
:100190008093F10080917B018093F10080917C013C
:1001A0008093F10080917D018093F10080917E0128
:1001B0008093F1008091E8008E7F8093E800809129
:1001C000E80080FFFCCF8091E80082FFFCCF8091A7
:1001D000E8008B7F8093E8008091E8008F77809320
:1001E000E80008958091E800877F8093E80080917F
:1001F000E80082FFFCCF8091F1008093780180912C
:10020000F100809379018091F10080937A018091CF
:10021000F10080937B018091F10080937C018091BB
:10022000F10080937D018091F10080937E018091A7
:10023000E8008B7F8093E8008091E8008F778093BF
:10024000E8008091E8008E7F8093E8008091E800CC
:1002500080FFFCCF209178013091790140917A01A3
:1002600050917B01569547953795279584E0220F4D
:10027000331F441F551F8A95D1F760E072E18AE76A
:1002800090E00E946408215030403093CD002093CC
:10029000CC0008958091F1008091F100613231F03D
:1002A000623259F0603229F080E008950E94B9006E
:1002B00002C00E94F20081E008958091E800877FEB
:1002C0008093E8008091E8008E7F8093E800809121
:1002D000E80080FFFCCF81E008958091E800877FEF
:1002E0008093E8008091E8008E7F8093E800809101
:1002F000E80080FFFCCF0895FF920F931F9309EE53
:1003000010E083E0F801808360E281EC0E945C02EF
:1003100081E0F801808360E281E80E945C0222E0D3
:10032000F22EF801F08264E280E80E945C02EAEEBC
:10033000F0E088E080831082F082108284E0808385
:1003400010821F910F91FF90089580917F018F5F20
:1003500080937F01089580918201882309F455C01C
:1003600080917F01823340F080918701882321F0C2
:1003700010927F010E94B3060E941906882341F063
:100380000E943B06992787FD90950E9492064C9A01
:100390008091C80085FF11C00E944706882349F458
:1003A0000CC00E946906992787FD90950E9432062D
:1003B0004F9A809188018823A1F780917F0184362C
:1003C00020F11D9904C080E091E00E940A07649921
:1003D00004C082E191E00E940A071E9904C083E2F2
:1003E00091E00E940A07659904C083E391E00E94AE
:1003F0000A071F9904C083E491E00E940A076299EA
:1004000004C081E591E00E940A0708950E941D063C
:100410008AB1806F8AB984B18F7184B985B1806ED9
:1004200085B98DB1877E8DB98EB180638EB96A989A
:10043000729AE2EEF0E080818460808369E676E083
:1004400082E996E00E94BE060895A89587EF84BFD2
:10045000E0E6F0E08081886180831082E1E6F0E0F0
:1004600080E8808310820E94140680E090E0089566
:1004700013BE83B7856083BF8895089513BE83B785
:10048000816083BF8895089513BE83B7836083BF5F
:100490008895089513BE83B7876083BF88950895B4
:1004A00013BE83B78D6083BF8895089513BE83B74D
:1004B0008F6083BF889508959091EB009160909331
:1004C000EB008093EC008091ED008270862B80938E
:1004D000ED008091ED0082608093ED008091EE0050
:1004E000881F8827881F08959091F40080E090FD70
:1004F00006C08F5F873011F09695F9CF80E00895A0
:10050000FB018093E90004C081918093F100415088
:100510008091E80085FF02C04423B1F7842F08953D
:10052000FB018093E90004C08091F1008193415068
:100530008091E80085FF02C04423B1F7842F08951D
:100540008093E900EBEEF0E0808180628083089583
:100550008091D8008F7B8093D8008091D90081FF53
:1005600021C01092E9008091EB0080FD1BC0109229
:10057000E9008091EB0081608093EB0082E0809342
:10058000EC008091ED00827080638093ED0080919B
:10059000ED0082608093ED008091EE00881F882737
:1005A000881F089580E00895089578940E94380285
:1005B00008951F920F920FB60F920BB60F9211244F
:1005C0002F933F934F935F936F937F938F939F935B
:1005D000AF93BF93EF93FF938091DA0080FF31C018
:1005E0008091D80080FF2DC08EEF8093DA0080913B
:1005F000D90080FF19C081E080938601809170014D
:10060000909171018260909371018093700180914B
:10061000E20088608093E2000E94C1058091E000C2
:100620008E7F8093E0000DC01092860110928201AF
:100630008091700190917101846090937101809319
:1006400070018091E10082FF09C08091E20082FF89
:1006500005C08BEF8093E1000E94A5018091E1002D
:1006600080FF1FC08091E20080FF1BC08EEF80934F
:10067000E1008091E20080618093E2008FEE809340
:10068000E1008091D80080628093D8008091700151
:1006900090917101806290937101809370010E942A
:1006A000D5028091E10084FF1AC08091E20084FFAE
:1006B00016C08091D8008F7D8093D8008FEE8093F4
:1006C000E1008091E2008F7E8093E20080917001D2
:1006D0009091710180649093710180937001809179
:1006E000E10085FF1AC08091E20085FF16C080916D
:1006F000E2008F7E8093E2008FED8093E100809195
:10070000E2008F7D8093E2008091700190917101F1
:10071000806890937101809370018091E10083FF64
:1007200012C08091E20083FF0EC087EF8093E1004A
:100730000E94A80280917001909171019160909344
:10074000710180937001FF91EF91BF91AF919F91E3
:100750008F917F916F915F914F913F912F910F906A
:100760000BBE0F900FBE0F901F9018950E94DD05D5
:100770000895E7EDF0E080818160808380818F7B48
:1007800080838081806880830E94B0050895DF9314
:10079000CF9300D0CDB7DEB79091F1009093770161
:1007A0006091F1006630F9F0673068F4613009F467
:1007B00002C1613008F46CC1633009F435C16530A1
:1007C00009F0BAC1BEC0693009F4DCC06A3020F457
:1007D000683009F0B1C199C06A3009F495C16B3035
:1007E00009F0AAC198C1903809F08DC01092720129
:1007F0006091F1008091F100813019F0823089F42C
:1008000006C082E18093830188E990E005C083E41B
:10081000809383018AEA90E090938501809384011C
:1008200005C00E94B700882309F48BC18091F100B4
:100830008091F1008091F10089838091F1008A8399
:100840008091E800877F8093E80029813A81809138
:10085000830190E08217930758F48F739070892B6F
:1008600021F481E08093720105C01092720102C0F0
:10087000209383012091840130918501409183016F
:1008800019C08091E80080FFFCCFF90190E00AC018
:10089000542F5150903449F09F5F84918093F10020
:1008A0003196452F9F01442399F78091E8008E7F70
:1008B0008093E800442359F08091E80082FFE1CF63
:1008C00020938401309385014093830106C02093D7
:1008D000840130938501109283018091E80082FDAC
:1008E00008C180917201813049F48091E80080FF55
:1008F000FCCF8091E8008E7F8093E8008091E80033
:1009000082FFFCCFF6C066E002C19038C1F480914E
:10091000E800877F8093E800809182018093F10056
:100920008091E8008E7F8093E8008091E8008F77C7
:100930008093E8008091E80082FFFCCFDAC068E095
:10094000E6C09923E9F49091E3008091F1008F775C
:100950009078892B8093E3008091E800877F8093D3
:10096000E8008091E8008E7F8093E8008091E800A5
:1009700080FFFCCF8091E30080688093E300EBC0B0
:1009800065E0C5C09923A9F49091F100923008F078
:10099000D8C08091E800877F8093E800909382011F
:1009A0008091E8008E7F8093E800892F0E947C016F
:1009B000D2C069E0ACC09330A8F5992309F4C1C056
:1009C000913009F4BEC08091F1009091F10088232C
:1009D00009F0B7C0E091F100EF77E093E900809172
:1009E000EB0080FF50C0EE23B1F08091EB008061FE
:1009F0008093EB0081E090E00E2E02C0880F991FDB
:100A00000A94E2F78093EA001092EA008091EB00EA
:100A100088608093EB001092E900F0E0ED58FE4F03
:100A2000108228C061E073C0933080F5913009F4E2
:100A300088C0923009F08FC08091F1009091F10050
:100A4000882309F07EC0E091F100EF7709F479C0C6
:100A5000E093E9008091EB0080FF15C08091EB00EE
:100A600080628093EB001092E900F0E0ED58FE4FB9
:100A700081E080838091E800877F8093E800809107
:100A8000E8008E7F66C01092E9005BC063E03FC063
:100A9000892F80588330B0F58091F1008091F1006A
:100AA000E091F100913829F0923859F0903809F02E
:100AB00048C08091E800877F8093E8001092F100A1
:100AC0000DC08091E800877F8093E800F0E0EF7729
:100AD000F070ED58FE4F80818093F1001092F1008C
:100AE0008091E8008E7F8093E8008091E80082FF8B
:100AF000FCCF8091E8008B7F8093E8008091E80034
:100B00008F7727C060E003C09138D9F06AE0892F61
:100B10000E944A0120C09130F1F48091E800877F63
:100B20008093E8008091E8008E7F8093E8008091B8
:100B3000E80080FFFCCF0FC0892F0E944A01882364
:100B400051F48091EB0080628093EB008091E8008B
:100B5000877F8093E8000F900F90CF91DF910895E9
:100B60007894E8EDF0E080818F76808380818069E1
:100B7000808380818F7B8083808181608083789473
:100B800008958EE089BD09B400FEFDCF8091D800A4
:100B90008F7D8093D8008091E20081608093E20095
:100BA0008091E20088608093E2000E94A802809118
:100BB000E0008E7F8093E00008958091D90080FF4F
:100BC00009C080918601882329F481E08093860101
:100BD0000E94C105809170019091710190FF10C039
:100BE00080917001909171019E7F9093710180932B
:100BF000700181E08093EA001092EA001092820175
:100C00001092E9008091E80083FF02C00E94C703B0
:100C1000089508950E94B6030E94AB01FBCF0E9485
:100C2000B9030E94060208950E940F060E940A0658
:100C300008958091C8008078089589E190E09093AC
:100C4000CD008093CC00E8ECF0E08081826080836E
:100C500086E08093CA00E9ECF0E0808188618083BF
:100C600081E00895282F8091C80085FFFCCF209354
:100C7000CE00822F08958091C80087FFFCCF80911D
:100C8000CE000895109287011092880108958091F6
:100C900088018823C9F482E08093E9008091E8000C
:100CA00082FF12C08091F3008091F200809388014E
:100CB000882351F48091E8008B7F8093E800809135
:100CC000E8008F778093E80080918801811181E0AE
:100CD000089582E08093E90080918801882319F4C7
:100CE0000E944706FBCF9091F100809188018150CE
:100CF00080938801882351F48091E8008B7F809352
:100D0000E8008091E8008F778093E800892F0895AC
:100D10008091E80090E025E0969587952A95E1F787
:100D200081700895282F81E08093E9008091E80088
:100D300085FFFCCF0CC081E08093E9008091E80042
:100D40008F778093E80010928701822F0895209377
:100D5000F100809187018F5F809387018091E80087
:100D600085FFE9CFF2CF81E08093E900E8EEF0E083
:100D700080818F7780831092870108950F931F934E
:100D8000CF93DF938C01EB01009731F4611571056E
:100D900019F420E030E038C06EE070E081E090E0CF
:100DA0000E943F07FC019C01009771F180E883835A
:100DB000209771F0D387C28781E88383809189016E
:100DC00090918A01892B21F4F0938A01E0938901A3
:100DD00001151105C9F01187008783818260838323
:100DE00080918B0190918C01892B71F4F0938C018F
:100DF000E0938B0180918D0190918E01892B21F4DC
:100E0000F0938E01E0938D01C901DF91CF911F9185
:100E10000F9108950F931F93CF93DF938C01E0916F
:100E20008B01F0918C01838181FF21C0C0E0D0E073
:100E30000DC0E0918B01F0918C0120853185BF01BF
:100E4000F9010995892B11F0CFEFDFEFF8018191BE
:100E50008F01882371F7E0918B01F0918C0120853F
:100E60003185BF018AE0F9010995892B11F0CFEF97
:100E7000DFEFCE01DF91CF911F910F9108950F9376
:100E80001F93CF93DF93689F8001699F100D789F18
:100E9000100D1124C8010E945B07EC01009729F096
:100EA000A80160E070E00E945D08CE01DF91CF9163
:100EB0001F910F910895CF93DF93BC01823091056C
:100EC00010F462E070E0A0919101B0919201ED0107
:100ED000E0E0F0E040E050E021C088819981861791
:100EE000970769F48A819B81309719F093838283F5
:100EF00004C09093920180939101FE0134C0681761
:100F0000790738F44115510519F08417950708F44D
:100F1000AC01FE018A819B819C01E9012097E9F6E1
:100F200041155105A9F1CA01861B970B049708F4D6
:100F3000BA01E0E0F0E02AC08D919C9111978417EE
:100F40009507F9F46417750781F412968D919C91B9
:100F50001397309719F09383828304C09093920182
:100F600080939101FD0132964CC0CA01861B970BFC
:100F7000FD01E80FF91F6193719302978D939C9384
:100F800040C0FD01828193819C01D9011097A1F697
:100F900080918F0190919001892B41F480916C0197
:100FA00090916D019093900180938F0140916E011B
:100FB00050916F014115510541F44DB75EB78091D5
:100FC0006A0190916B01481B590B20918F01309160
:100FD0009001CA01821B930B8617970780F0AB0123
:100FE0004E5F5F4F8417950750F0420F531F509389
:100FF000900140938F01F9016193719302C0E0E089
:10100000F0E0CF01DF91CF910895CF93DF93009768
:1010100009F450C0EC0122971B821A82A091910121
:10102000B0919201109709F140E050E0AC17BD0774
:1010300008F1BB83AA83FE0121913191E20FF31FD6
:10104000AE17BF0779F48D919C911197280F391F26
:101050002E5F3F4F3983288312968D919C91139771
:101060009B838A834115510571F4D0939201C093FB
:10107000910120C012968D919C911397AD0100971C
:1010800011F0DC01D3CFFA01D383C28321913191D6
:10109000E20FF31FCE17DF0769F488819981280FCB
:1010A000391F2E5F3F4FFA01318320838A819B8154
:1010B00093838283DF91CF910895DC0101C06D930A
:1010C00041505040E0F70895A1E21A2EAA1BBB1B25
:1010D000FD010DC0AA1FBB1FEE1FFF1FA217B30704
:1010E000E407F50720F0A21BB30BE40BF50B661F1A
:1010F000771F881F991F1A9469F7609570958095DE
:1011000090959B01AC01BD01CF010895F894FFCFEC
:1011100053656C6563742050726573736564202138
:101120000D0052696768742050726573736564209E
:10113000210D004C656674205072657373656420E0
:10114000210D00446F776E205072657373656420C3
:10115000210D005570205072657373656420210D58
:101160000048656C6C6F2066726F6D204154393099
:1011700055534258585820210D002000930100007B
:00000001FF
